:040000008A01082841
:080008000B1109006E288F287E
:1000100083160730831603139F0083128316C030A4
:1000200081008312F6010130F500043076020319D5
:100030005528F7017508F50083168316031385010B
:100040008312750883128500F0017608013E0318BB
:10005000F00AF6007508F000700DFE39F500FE306C
:10006000F40008307702031915288316831603134A
:1000700086018312740883128600FA30F10006208C
:100080008A110A127408F000700DFE39F400F001B4
:100090007408013E0318F00AF400F0017708013EED
:1000A0000318F00AF700312815280F30F5008316E1
:1000B0008316031385018312750883128500F401EA
:1000C000831683168601831274088312860001301A
:1000D000F30007208A110A1212286D28DF30F2007F
:1000E0000000000000000000000000000000000010
:1000F0000000000000000000000000000000000000
:1001000000000000000000000000000000000000EF
:10011000F20B75280000F10B6E2800000800FA3081
:10012000F10006208A110A12FA30F10006208A1125
:100130000A12FA30F10006208A110A12FA30F10090
:0C01400006208A110A12F30B8F28080019
:04400E002A3FFC3F0A
:00000001FF
